:020000040800F2
:1000000000500020093E00085D0700085F07000857
:10001000610700086307000865070008000000008A
:10002000000000000000000000000000670700085A
:1000300069070008000000006B0700086D07000852
:10004000513E0008513E0008513E0008513E000854
:10005000513E0008513E0008513E0008513E000844
:10006000513E0008513E0008513E0008513E000834
:10007000513E0008513E0008513E0008E9010008C9
:10008000513E0008513E0008513E0008513E000814
:1000900075070008513E0008513E0008513E000817
:1000A000513E0008513E0008513E0008513E0008F4
:1000B000513E0008513E0008513E0008513E0008E4
:1000C000513E0008513E0008513E0008513E0008D4
:1000D000513E0008513E0008513E0008513E0008C4
:1000E000513E0008513E0008513E0008000000004B
:1000F0000000000000000000000000000000000000
:0C01000000000000000000005FF808F1A3
:10010C000348044B834202D0034B03B1184770479A
:10011C007C0100207C010020000000000548064BFB
:10012C001B1AD90F01EBA301491002D0034B03B1E9
:10013C00184770477C0100207C0100200000000063
:10014C0010B5064C237843B9FFF7DAFF044B13B113
:10015C000448AFF300800123237010BD7C01002004
:10016C0000000000AC3E000808B5054B1BB105496A
:10017C000548AFF30080BDE80840FFF7CFBF00BFD4
:10018C000000000080010020AC3E0008044B5A6CBB
:10019C0042F400425A641A6A42F001021A62704731
:1001AC00002C01400C4B1A6822F001021A601A6AEA
:1001BC0022F001021A62D862596300225A621A6A4A
:1001CC0042F001021A625A6942F001025A611A683D
:1001DC0042F001021A607047002C0140704700B5D4
:1001EC0000F00700C0F1070CBCF1040F28BF4FF062
:1001FC00040C031D062B0FD9C31E4FF0FF3E0EFA45
:10020C000CF021EA000199400EFA03FE22EA0E02DC
:10021C0041EA02005DF804FB0023EEE710B4836BA7
:10022C00C3F301530133846BCB1ADBB20333DBB260
:10023C0003EB83031F21994024EA010402F01F02FF
:10024C009A401443846310BC7047000010B44029DA
:10025C0010D007D804290FD010290FD001290FD1A5
:10026C00002210E0B1F5807F0CD0B1F5806F19D170
:10027C00052208E0032206E0012204E0022202E04B
:10028C00062200E004221830074B995C4358074CB7
:10029C0014F802C0042202FA0CF223EA02034350BF
:1002AC0010BC70470622EEE7CC3E0008C43E0008A6
:1002BC0000B583B00E4B5A6942F001025A615B697A
:1002CC0003F001030193019B0A4BD86800221146ED
:1002DC00C0F30220FFF783FF0001C0B2064B83F886
:1002EC000F034FF400421A6003B05DF804FB00BF2B
:1002FC000010024000ED00E000E100E0F0B589B034
:10030C000024039404940594069407941B4B9A6957
:10031C0042F010029A619A6902F010020292029A5B
:10032C009A6942F020029A619A6902F020020192C5
:10033C00019A9A6942F004029A619B6903F00403E2
:10034C000093009B0E484FF4005343610D4D062360
:10035C006B610D4B0393012704970226059603A9A5
:10036C0000F03AFC40F2066303930497059606945A
:10037C0003A9284600F030FC09B0F0BD0010024083
:10038C0000100140000801402000200430B50C3062
:10039C0001F0007E4FF0007393FAA3F3B3FA83F3EA
:1003AC002EFA03FE50F82E4001F0F8714FF0F8735E
:1003BC0093FAA3FCBCFA8CFC21FA0CFC072505FA79
:1003CC000CFC24EA0C0C93FAA3F3B3FA83F3D94094
:1003DC008A404CEA020240F82E2030BDF0B595B0B0
:1003EC0000241294139411940C940D940E940F9465
:1003FC001094089409940A940B940394049405940F
:10040C0006940794384B9A6942F400729A619A697F
:10041C0002F400720292029A9A6942F004029A6102
:10042C009B6903F004030193019B41F618030393AA
:10043C0003A92E4800F0D0FB12944FF48073139351
:10044C002B4D12A9284602F0E3FC119411A9284661
:10045C0002F0C2FC4FF460230C930D940E940F9495
:10046C0010940CA9284602F0E7FC4FF4E0430893E3
:10047C004FF4801309930A940B9408A9284602F0B0
:10048C0006FD1C4E324601212846FFF7C7FE2246C8
:10049C0031462846FFF77AFF4FF4405696FAA6F3FA
:1004AC00154AD2F814346FF30B03C2F81434134FFB
:1004BC003A4641F202112846FFF7B0FE2246394671
:1004CC002846FFF763FF96FAA6F6B6FA86F64FF4BF
:1004DC008053F3400A4951F823206FF30B0241F883
:1004EC00232015B0F0BD00BF0010024000080140F1
:1004FC000024014003009002002001400400C002CF
:10050C0014240140F0B59BB0002415941694179454
:10051C001894199420252A4621460DA803F0B8FCFE
:10052C000794089409940A940B940C9402940394E1
:10053C00049405940694444EB36943F40063B36188
:10054C00B36903F400630193019B404B9A6D22F451
:10055C00804222F0100242F010029A659A6D22F449
:10056C0040529A659A6D22F020029A659A6D22F09B
:10057C0040029A659A6D42F080029A659A6D22F457
:10058C00407242F400729A659A6D22F4406242F411
:10059C0000629A654FF49653ADF854301695642367
:1005AC001793189401271997294D15A9284603F07C
:1005BC00B5FB2B6823F080032B60AB6823F48043DE
:1005CC0023F00703AB6030230D930E940F94462356
:1005DC00109311941294139414940DAA394628462E
:1005EC0003F0D4FB39462846FFF730FE6B6823F046
:1005FC0070036B60AB6823F08003AB6007940894C6
:10060C0009948DF82840ADF82A404FF400530B9311
:10061C000C9407A9284603F0D7FBB36943F00403F5
:10062C00B361B36903F004030093009B094B02937D
:10063C000923039302230493059402A9064800F0AE
:10064C00CBFA1BB0F0BD00BF00100240000002400E
:10065C00002C0140010001040008014072B6FEE7C5
:10066C0008B52B4A136823F0070343F0010313600A
:10067C00274B1B6803F00703012BF9D1254A13689C
:10068C0043F480331360234B1B6813F4003FFAD000
:10069C00204A536823F47C1343F488135360136883
:1006AC0043F0807313601B4B1B6813F0007FFAD070
:1006BC00184B5A6822F0F0025A605A6822F4E06231
:1006CC0042F480625A605A6822F460525A605A6846
:1006DC0022F0030242F002025A600E4B5B6803F0F8
:1006EC000C03082BF9D10C4802F0C0FA0F2002F0D1
:1006FC00C3FA58B9074A536823F4404343F4804380
:10070C005360536843F48003536008BDFFF7A6FFA2
:10071C000020024000100240006CDC0208B502F020
:10072C00D1FAFFF79DFFFFF7E9FDFFF7C1FDFFF7DA
:10073C0055FE00F043F8FFF7E5FEFFF727FD4FF4F9
:10074C00FA7002F07DFA4FF4FA7002F079FAFAE7D7
:10075C00FEE7FEE7FEE7FEE7FEE7704770477047EF
:10076C0008B502F0C1FA08BD08B5024801F0AFF8AF
:10077C0008BD00BF5C0E002082B00E4B9A6942F09F
:10078C0001029A619A6902F001020092009ADA69F8
:10079C0042F08052DA61DB6903F080530193019BD4
:1007AC00054A536823F0E06343F00073536002B0D2
:1007BC00704700BF001002400000014008B5002245
:1007CC000F49104802F08BFB70B90F490D4802F02D
:1007DC009DFB60B90D490B4803F0A1F950B90948CC
:1007EC0002F09BFB48B908BDFFF738FFEDE7FFF7B8
:1007FC0035FFEFE7FFF732FFF1E7FFF72FFFF2E7E7
:10080C0000000020980100206C0000205000002007
:10081C0012230B80004870471C00002004230B801F
:10082C000048704730000020002393421ED200B5D0
:10083C0010E00CF1370C01F813C000014FEA430C27
:10084C000CF1010C4FF0000E01F80CE00133DBB29F
:10085C00934209D24FEA107CB0F1204FE9D20CF14F
:10086C00300C01F813C0E8E75DF804FB704700009A
:10087C0038B50B4BD3F8E807D3F8EC47D3F8F0377F
:10088C00C01800D138BD074D0822A91CFFF7CCFFBA
:10089C00042205F112012046FFF7C6FFF2E700BF64
:1008AC0000F0FF1F3400002008B51A230B80FFF75F
:1008BC00DFFF014808BD00BF3400002008B50A4620
:1008CC0028B90549054802F080FF034808BD0249D4
:1008DC00024802F07AFFF8E75C040020D43E0008DE
:1008EC0010B50A46034C2146034802F06EFF204621
:1008FC0010BD00BF5C040020EC3E000808B50A46A1
:10090C0028B90549054802F060FF034808BD0249B3
:10091C00024802F05AFFF8E75C040020003F000890
:10092C0008B50A4628B90549054802F04EFF0348A8
:10093C0008BD0249024802F048FFF8E75C040020B9
:10094C000C3F0008002070470020704738B5044663
:10095C00064D0146284603F0F1F8284603F0F4F85A
:10096C0061782078FFF71EFC002038BD980100202C
:10097C0010B5064C00220649204603F0D7F805496D
:10098C00204603F0DBF8002010BD00BF98010020CA
:10099C005C0600205C0A0020022805D8DFE800F085
:1009AC0005040200012070470220704702680E4BBC
:1009BC009A4200D0704700B583B003F5DA33DA6998
:1009CC0042F40002DA61DB6903F400030193019B3A
:1009DC0000221146142002F0A5F9142002F0DAF9D5
:1009EC0003B05DF804FB00BF005C004008B500F5E7
:1009FC002C71D0F8EC0202F0A8FA08BD08B501EB96
:100A0C00810300EBC303D3F87C21D0F8EC0202F095
:100A1C00C9FA08BD08B501EB810300EBC303DA6B1F
:100A2C00D0F8EC0202F004FB08BD08B5D0F8EC02DB
:100A3C0002F0A5FB08BD10B504468368022B09D152
:100A4C000121D4F8EC0202F083FBD4F8EC0202F0A2
:100A5C0057FB10BDFFF702FEF2E7000010B504468D
:100A6C00D0F8EC0202F077FBA36923B1024A1369B8
:100A7C0043F00603136110BD00ED00E008B5D0F89B
:100A8C00EC0202F071FB08BD10B504461D48C0F81D
:100A9C00EC42C4F8C0021C4B0360082343600223E1
:100AAC00836000238361C361036200F0AEF930BB45
:100ABC00182300221146D4F8C00201F00FF9582374
:100ACC0000228021D4F8C00201F008F9C0230022D2
:100ADC008121D4F8C00201F001F94FF4887300228F
:100AEC000121D4F8C00201F0F9F84FF48073002210
:100AFC008221D4F8C00201F0F1F8002010BDFFF7FC
:100B0C00ADFDD5E75C0E0020005C004008B5D0F8C8
:100B1C00C00200F002FAFFF73FFF08BD08B594468B
:100B2C001A466346D0F8C00200F0A9FFFFF734FF65
:100B3C0008BD08B5D0F8C00200F0DFFFFFF72CFFAE
:100B4C0008BD08B5D0F8C00201F051F8FFF724FF3A
:100B5C0008BD08B5D0F8C00201F085F8FFF71CFFFE
:100B6C0008BDD0F8C03211F0800F08D101F07F0120
:100B7C0001EB810103EBC10191F86A01704701F0AF
:100B8C007F01013101EB810103EBC10188787047D2
:100B9C0008B5D0F8C00200F086FEFFF7FDFE08BDD8
:100BAC0008B5D0F8C00201F000F8FFF7F5FE08BD5B
:100BBC0008B5D0F8C00200F0D2FFFFF7EDFE08BD7B
:100BCC0008B5D0F8C00200F0E7FF08BD0048704738
:100BDC004C110020704770470B68C3F30F2C9CFA24
:100BEC00ACF2B2FA82F276E0A2F108044FF00113F3
:100BFC00A34043F080634C68082C2CD01D0E93FA54
:100C0C00A3F4B4FA84F4A4004FF00F0E0EFA04F41B
:100C1C00465926EA040493FAA3FEBEFA8EFE4FEA66
:100C2C008E0E4E6806FA0EFE44EA0E0444514C68D1
:100C3C00012C1ED0092C1CD001323CFA02F347D0F7
:100C4C000123934013EA0C0FF6D0072ACCD840F2BC
:100C5C0001139340CFE70D69C6681C0A26EA1326D8
:100C6C0094FAA4F4B4FA84F405FA04F43443C4609A
:100C7C00C4E74FEA136E50F80E4093FAA3F5B5FA99
:100C8C0085F5AD00032606FA05F524EA050493FA6A
:100C9C00A3F5B5FA85F5AD008E6806FA05F5254382
:100CAC0040F80E50CC6893FAA3F6B6FA86F6B60066
:100CBC00042707FA06F625EA060593FAA3F3B3FA16
:100CCC0083F39B0004FA03F32B4340F80E30B3E795
:100CDC000020F0BD01323CFA02F306D00123934010
:100CEC0013EA0C0FF6D0F0B5AFE70020704738B51B
:100CFC0012F4804F44D00468B4F850309BB291F891
:100D0C0000C003EBCC03023304EB4303B3F8004401
:100D1C00C4F309048B69A34228D31B1B8B618B6919
:100D2C007BB9056835F82C309BB223F4804323F053
:100D3C00700383F4005343F4004343F0800325F81D
:100D4C002C3012F0400F0ED002680D7832F825309E
:100D5C009BB223F4E04323F0700343F4004343F0CD
:100D6C00C00322F8253024B9204638BD00238B61FE
:100D7C00D5E723460A894969006801F049FFF3E782
:100D8C000468B4F850309BB291F800C003EBCC036C
:100D9C00063304EB4303B3F80044C4F309048B6932
:100DAC00A3422FD31B1B8B618B697BB9056835F86C
:100DBC002C309BB223F4804323F0700383F4005354
:100DCC0043F4004343F0800325F82C3012F0400F1D
:100DDC000FD1026891F800C032F82C309BB223F48A
:100DEC00E04323F0700343F4004343F0C00322F8C4
:100DFC002C30002CB8D023464A894969006801F090
:100E0C0007FFB1E700238B61CEE770B586B00028F1
:100E1C0000F08180044690F8A932EBB1032384F8EA
:100E2C00A932206800F086FF254655F8106BEC4679
:100E3C000FCDACE80F002B68CCF80030231D0ECB87
:100E4C00304600F067FF054658B1022384F8A932FA
:100E5C000125284606B070BD80F8A832FFF7A6FD24
:100E6C00DCE70021206800F06FFF2B4616E05A1CCF
:100E7C0002EB820104EBC1010120487002EB8201FC
:100E8C0004F8313004EBC1000021C17003EB830086
:100E9C0004EBC0008163C1630164D3B261688B420F
:100EAC00E5D316E005EB850304EBC303002283F8BE
:100EBC00692183F8685183F86B21C3F87821C3F852
:100ECC007C2105EB850304EBC303C3F880210135BA
:100EDC00EDB2A942E6D8254655F8106BEC460FCD7D
:100EEC00ACE80F002B68CCF80030231D0ECB30463D
:100EFC0000F02CFF054620B1022384F8A93201250D
:100F0C00A7E7002384F82430012384F8A932206851
:100F1C0001F07BFA9DE701259BE738B590F8A832E4
:100F2C00012B11D00446012580F8A852006800F06E
:100F3C00F8FE29462046FFF74EFE206801F063FAC2
:100F4C00002084F8A80238BD0220FCE770B50546E5
:100F5C000C46164612F0400F00F00E810268B2F8F3
:100F6C0050309BB2097803EBC103023302EB43030D
:100F7C00B3F80024C2F30902A36993424ED99B1A19
:100F8C00A361A369002B66D16378002B49D12B6830
:100F9C00B3F8502092B2134403EB0111B1F80434AE
:100FAC00C3F30903A1F80434B1F804346FEA4343E2
:100FBC006FEA53439BB2A1F804342B686278002A81
:100FCC003CD1B3F8502092B21344227803EB0213B5
:100FDC00B3F80C24C2F30902A3F80C24B3F80C24C4
:100FEC006FEA42426FEA524292B2A3F80C24217883
:100FFC002846FFF70FFD16F4804F41D02A68217860
:10100C0032F821309BB223F4E04323F0700343F415
:10101C00404343F0800322F8213031E00023A361E8
:10102C00AFE7012BC9D12B68B3F8502092B213440F
:10103C0003EB01110023A1F80434BEE7012AD6D139
:10104C00B3F8502092B21344227803EB021300221F
:10105C00A3F80C24CBE716F4804F0DD0286830F899
:10106C0021309BB223F4E04323F0700343F440435C
:10107C0043F0800320F8213094F82430012B12D057
:10108C002A68217832F821309BB223F4E04323F014
:10109C00400383F0300343F4004343F0800322F811
:1010AC002130002070BD636913446361E36913440C
:1010BC00E361216A2369994224D3C91A21626278B7
:1010CC00002A44D12A68B2F8501089B20A44217817
:1010DC0002EB0112B2F80414C1F30901A2F80414D2
:1010EC003E2B1BD9580913F01F0F00D10138B2F851
:1010FC00041489B2800280B2014341F40041A2F889
:10110C00041426E021B9002384F824301346D6E7D2
:10111C00002384F8243023620B46D0E74BB9B2F895
:10112C0004146FEA41416FEA514189B2A2F80414E8
:10113C000FE0590813F0010F00D00131B2F804048C
:10114C0080B2890289B20143A2F8041401E0012A99
:10115C0006D09BB222896169286801F05EF98FE79D
:10116C002A68B2F8501089B20A44217802EB0112B5
:10117C0099B2A2F80414ECE70268B2F850309BB2B2
:10118C00097803EBC103063302EB4303B3F80024E5
:10119C00C2F30902A36993424FD39B1AA361A369BB
:1011AC00002B67D16378002B4AD12B68B3F8502001
:1011BC0092B2134403EB0111B1F80434C3F30903E5
:1011CC00A1F80434B1F804346FEA43436FEA534393
:1011DC009BB2A1F804342B686278002A3DD1B3F895
:1011EC00502092B21344227803EB0213B3F80C2470
:1011FC00C2F30902A3F80C24B3F80C246FEA4242A0
:10120C006FEA524292B2A3F80C2421782846FFF7D9
:10121C0001FC16F4804F7FF433AF2A68217832F842
:10122C0021309BB223F4E04323F0700343F440439A
:10123C0043F0800322F8213022E70023A361AEE7BC
:10124C00012BC8D12B68B3F8502092B2134403EB96
:10125C0001110023A1F80434BDE7012AD5D1B3F85C
:10126C00502092B21344227803EB02130022A3F80D
:10127C000C24CAE716F4804F0DD1286830F82130C1
:10128C009BB223F4E04323F0700343F4404343F058
:10129C00800320F8213094F82430012B7FF4F0AE39
:1012AC00636913446361E3691344E361216A23694D
:1012BC00994224D3C91A21622A686178002943D142
:1012CC00B2F8501089B20A44217802EB0112B2F83C
:1012DC000C14C1F30901A2F80C143E2B1BD95809AC
:1012EC0013F01F0F00D10138B2F80C1489B2800230
:1012FC0080B2014341F40041A2F80C1426E021B95C
:10130C00002384F824301346D6E70023236284F8A4
:10131C0024300B46D0E74BB9B2F80C146FEA4141BC
:10132C006FEA514189B2A2F80C140FE0590813F07E
:10133C00010F00D00131B2F80C0480B2890289B2DD
:10134C000143A2F80C1401E0012906D09BB262897A
:10135C006169286801F061F892E6B2F8501089B220
:10136C000A44217802EB011299B2A2F80C14EDE7B1
:10137C002DE9F04105462868B0F8443013F4004FCD
:10138C0000F08E82B0F84440A3B214F00F0440F089
:10139C00E28013F0100F6BD003889AB213F4006F35
:1013AC0040F09D8012F4004FE5D0038823F07003C9
:1013BC001B051B0D43F0800303802868B0F85030E8
:1013CC009BB295F8682103EBC203063300EB430391
:1013DC00B3F80034C3F30903C5F884318BB1D5F8E5
:1013EC007C1171B1B5F86E2101F012FCD5F8842195
:1013FC00D5F87C311344C5F87C3100212846FFF721
:10140C00FDFA2A68138899B213F4006FB3D101F472
:10141C004051B1F5405FAED0B2F850309BB21A4497
:10142C00B2F80C34C3F30903A2F80C34D5F87831B4
:10143C003E2B77D9590913F01F0F00D10139B2F89F
:10144C000C349BB2890289B20B4343F40043A2F8DB
:10145C000C342A6813889BB223F4804323F0700366
:10146C0083F4405343F4004343F08003138082E73A
:10147C0003889BB223F4E14323F070036FEA4343E8
:10148C006FEA53439BB203802A68B2F850309BB288
:10149C0095F8281003EBC103023302EB4303B3F8B6
:1014AC000034C3F309036B64EA6B1344EB63002150
:1014BC002846FFF7AFFA95F82430002B3FF45BAFCA
:1014CC002B6C002B7FF457AF95F824302A6843F02F
:1014DC008003A2F84C30002385F824304BE7B0F899
:1014EC0050309BB295F8682103EBC203063300EB36
:1014FC004303B3F80034C3F30903C5F88431B5F8DA
:10150C006E2105F52C7101F083FB2A68138823F0FA
:10151C0070031B051B0D43F0800313802846FFF757
:10152C0065FA28E74BB9B2F80C346FEA43436FEA1B
:10153C0053439BB2A2F80C348BE7590813F0010FFC
:10154C0000D00131B2F80C3498B28B029BB2034339
:10155C00A2F80C347DE730F824309EB213F4004F1F
:10156C004CD116F0800F3FF406AF621C02EB8201E7
:10157C0005EBC101286830F824309BB223F4E14319
:10158C0023F070036FEA43436FEA53439BB220F896
:10159C002430CB78012B00F0F28016F4807F40F0E1
:1015AC007A812868B0F850309BB2621C02EB820240
:1015BC0015F8326003EBC603023300EB4303B3F8B8
:1015CC000034C3F3090304EB840205EBC202126C72
:1015DC009A4240F24C8104EB840705EBC707D21A00
:1015EC003A6404EB840205EBC202126C002A40F050
:1015FC00458131462846FFF70DFABCE630F8243019
:10160C0023F070031B051B0D43F0800320F82430DE
:10161C0004EB8401C90001F5B47105EB010804EB7E
:10162C00840305EBC30393F87431002B42D1286873
:10163C00B0F850309BB204EB840205EBC20292F876
:10164C00682103EBC203063300EB4303B3F80074C9
:10165C00C7F3090717BB04EB840305EBC303D3F8EB
:10166C0084213A44C3F88421D3F87C213A44C3F84A
:10167C007C21D3F880313BB104EB840305EBC3032D
:10168C00D3F878319F4275D204EB840305EBC30386
:10169C0093F868112846FFF7B1F962E704EB84016F
:1016AC0005EBC1013B46B1F86E21D1F87C1101F07C
:1016BC00AFFAD0E704EB840305EBC30393F86B316B
:1016CC00022B35D0296804EB840205EBC20292F898
:1016DC00680131F820309BB223F4E04323F070030F
:1016EC0043F4004343F0C00321F82030286892F8FB
:1016FC00682130F8223013F4804F20D0B0F85030ED
:10170C009BB203EBC203023300EB4303B3F8007448
:10171C00C7F30907002F9ED004EB840105EBC10130
:10172C003B46B1F87021D1F87C1101F071FA92E7C7
:10173C00324641462846FFF7DAFA07468BE7B0F8FF
:10174C0050309BB203EBC203063300EB4303B3F8F8
:10175C000074C7F30907002F3FF47DAF04EB84013D
:10176C0005EBC1013B46B1F87221D1F87C1101F0B7
:10177C004FFA70E74146286800F063FEF1E604EB8F
:10178C00840305EBC30300221A6493F83430FBB1D5
:10179C0016F0400F37D04B781BBB2B68B3F850209A
:1017AC0092B21344621C02EB820215F8322003EB56
:1017BC000213B3F80424C2F30902A3F80424B3F807
:1017CC0004246FEA42426FEA524292B2A3F8042414
:1017DC00013404EB840415F834102846FFF71AF989
:1017EC00C9E5012BF4D12B68B3F8502092B2134405
:1017FC00621C02EB820215F8322003EB021300226A
:10180C00A3F80424E4E72A68631C03EB830305EBC9
:10181C00C3035B78D3B9B2F850309BB21344621C4B
:10182C0002EB820215F8322003EB0213B3F80C24FE
:10183C00C2F30902A3F80C24B3F80C246FEA424259
:10184C006FEA524292B2A3F80C24C1E7012BBFD12C
:10185C00B2F850309BB21344621C02EB820215F8B2
:10186C00322003EB02130022A3F80C24B0E704EBA4
:10187C00840205EBC20200271764B2E604EB840273
:10188C0005EBC202D66B1E44D663546C23445364DE
:10189C0000F0D7FD6FE532462846FFF757FB6AE5A7
:1018AC000020BDE8F08190F8A832012B0DD010B5C6
:1018BC000446012380F8A83280F82410006800F058
:1018CC009CFD002084F8A80210BD0220704710B5C2
:1018DC0084B00446006800F09AFD10F4004F20D14B
:1018EC0010F4806F21D110F4804F2FD110F4005FD1
:1018FC0037D110F4805F3ED110F4006F40F0878038
:10190C0010F4007F40F0AE8010F4807F27D0226866
:10191C00B2F844309BB223F480739BB2A2F84430EB
:10192C001DE02046FFF724FD19E02268B2F8443090
:10193C009BB223F480639BB2A2F844302046FFF79D
:10194C007AF800212046FFF7AEFF08E02268B2F8D3
:10195C0044309BB223F480439BB2A2F8443004B0D1
:10196C0010BD2268B2F844309BB223F400539BB2F2
:10197C00A2F84430F3E72268B2F840309BB223F06F
:10198C0004039BB2A2F840302268B2F840309BB2FC
:10199C0023F008039BB2A2F840302046FFF76EF804
:1019AC002268B2F844309BB223F480539BB2A2F865
:1019BC004430D4E7226832F8231004AA02EB430225
:1019CC0022F8101C0133DBB2072BF3D92268B2F8D2
:1019DC0040309BB243F00103A2F840302268B2F8C9
:1019EC0040309BB223F001039BB2A2F84030236835
:1019FC00B3F8442012F4806FF9D0B3F8442092B2BB
:101A0C0022F4806292B2A3F8442000230BE000235E
:101A1C00DAE7226804A901EB430131F8101C22F823
:101A2C0023100133DBB2072BF3D92268B2F8403014
:101A3C009BB243F00803A2F840302268B2F844305D
:101A4C009BB223F400639BB2A2F844302268B2F834
:101A5C0040309BB243F00403A2F840302046FEF71E
:101A6C00FDFF7CE72268B2F844309BB223F400738C
:101A7C009BB2A2F844302046FEF7D7FF6FE710B5B3
:101A8C000446084611F0800F25D101F0070C0CEB31
:101A9C008C01C90001F5B47E04EB0E010CEB8C0C2F
:101AAC0004EBCC0C4FF0000E8CF869E100F0070051
:101ABC0008700A61CB70022B1AD094F8A832012B53
:101ACC0019D0012384F8A832206800F050F90020C6
:101ADC0084F8A80210BD01F0070C0CF1010C0CEB02
:101AEC008C0104EBC1014FF0010E81F801E0DDE740
:101AFC0000230B71E1E70220ECE710B504460B461E
:101B0C0011F0800F1FD101F0070202EB8201C90016
:101B1C0001F5B471014402EB820200EBC202002019
:101B2C0082F8690103F007030B7094F8A832012BBB
:101B3C0013D0012384F8A832206800F0FDFA0020AD
:101B4C0084F8A80210BD01F00702013202EB8201F9
:101B5C0000EBC10101204870E4E70220F2E710B568
:101B6C0001F0070C0CEB8C01C90001F5B4710CEB06
:101B7C008C0E00EBCE0ECEF87C21CEF880310024FA
:101B8C00CEF884418EF869418EF868C10144006832
:101B9C0000F057FC204610BD01F0070101EB81015C
:101BAC0000EBC101D1F88401704738B501F007048E
:101BBC0004F1010C0CEB8C0104EB840E00EBCE0E4B
:101BCC00CEF83C20CEF8403001228EF84C20CEF8D6
:101BDC0048300025CEF8445000EBC1035A7000F891
:101BEC0031401946006800F02CFC284638BD38B549
:101BFC0001F007054268954231D804460B4611F0B6
:101C0C00800F1ED101EB8101C90001F5B4710144B3
:101C1C0003EB830300EBC303002283F86921012348
:101C2C008B700D7094F8A832012B1AD0012384F814
:101C3C00A832206800F06BFB5DB1002084F8A8028C
:101C4C0038BD6B1C03EB830100EBC10101224A7010
:101C5C00E5E704F52C71206800F0DDFBEDE70120D1
:101C6C00EEE70220ECE70B4601F00F0142689142CF
:101C7C0030D810B5044613F0800F21D103F00702C1
:101C8C0002EB8201C90001F5B471014402EB82023E
:101C9C0000EBC202002082F8690100228A7003F076
:101CAC0007030B7094F8A832012B15D0012384F88C
:101CBC00A832206800F050FB002084F8A80210BD68
:101CCC0003F00702013202EB820100EBC10101209B
:101CDC004870E2E7012070470220F0E711F0800F16
:101CEC000BD001F00701013101EB810100EBC101C7
:101CFC0052B90A73CB800020704701EB8101C900F7
:101D0C0001F5B4710144F3E701220A730B811B0C3A
:101D1C004B81F0E784B001A880E80E00002004B0ED
:101D2C00704703460020A3F844004FF43F42A3F849
:101D3C0040207047B0F8403023F47C535B045B0CBC
:101D4C00A0F84030002070470020704784B08446D3
:101D5C0001A880E80E000123ACF840300020ACF85C
:101D6C004000ACF84400ACF8500004B0704710B51B
:101D7C00034691F800C030F82C2092B222F4EC42C9
:101D8C0022F0700292B2C878032861D8DFE800F024
:101D9C00555C0258002048F2800E42EA0E0223F8ED
:101DAC002C2091F800C033F82C2092B222F4E0429F
:101DBC0022F070024CEA020242EA0E0223F82C20B6
:101DCC000A7B002A40F0DC804A78002A51D0B3F814
:101DDC00502092B21A440C7802EB0412B1F806C0EF
:101DEC004FEA5C0C4FEA4C0CA2F800C40C7833F8A8
:101DFC00242012F0400F0CD033F8242092B222F49D
:101E0C00E04222F0700242F4004242F0C00223F899
:101E1C002420CA78012A1DD0097833F8212092B2E7
:101E2C0022F4E04222F0400282F0200242F400420E
:101E3C0042F0800223F8212017E142F40072AAE755
:101E4C0042F4C0620020A6E742F480620020A2E7C0
:101E5C000120A0E7097833F8212092B222F4E04265
:101E6C0022F0400242F4004242F0800223F821208A
:101E7C00FBE0B3F8502092B21A440C7802EB041237
:101E8C00B1F806C04FEA5C0C4FEA4C0CA2F808C43F
:101E9C00B3F8502092B21A440C7802EB0412B2F848
:101EAC000CC4CCF3090CA2F80CC40C693E2C39D927
:101EBC004FEA541E14F01F0F01D10EF1FF3EB2F881
:101ECC000CC41FFA8CFC4FEA8E2E1FFA8EFE4CEAC5
:101EDC000E0C4CF4004CA2F80CC40C7833F82420F3
:101EEC0012F4804F0CD033F8242092B222F4E0424A
:101EFC0022F0700242F4404242F0800223F8242087
:101F0C00097869BB33F8212092B222F4804222F086
:101F1C00700282F4405242F4004242F0800223F8F4
:101F2C002120A2E04CB9B2F80C446FEA44446FEAA9
:101F3C005444A4B2A2F80C44CFE74FEA540C14F06A
:101F4C00010F01D00CF1010CB2F80C44A4B24FEA11
:101F5C008C2C1FFA8CFC44EA0C0CA2F80CC4BCE7C9
:101F6C0033F8212092B222F4804222F0700282F4E3
:101F7C00005242F4004242F0800223F8212074E027
:101F8C00CA78022A72D00C7833F8242092B222F448
:101F9C00E24222F0700242F4004242F0800223F846
:101FAC002420B3F8502092B21A4491F800C002EBEE
:101FBC000C12B1F808C04FEA5C0C4FEA4C0CA2F8BA
:101FCC0000C4B3F8502092B21A4491F800C002EB4E
:101FDC000C12B1F80AC04FEA5C0C4FEA4C0CA2F898
:101FEC0008C44A78002A50D10C7833F8242012F413
:101FFC00804F0CD033F8242092B222F4E04222F02D
:10200C00700242F4404242F0800223F824200C7803
:10201C0033F8242012F0400F0CD033F8242092B265
:10202C0022F4E04222F0700242F4004242F0C0027C
:10203C0023F8242091F800C033F82C2092B222F41B
:10204C00804222F0700282F4405248F28004224313
:10205C0023F82C20097833F8212092B222F4E042A4
:10206C0022F04002224323F8212010BD0C7833F8D3
:10207C00242092B222F4E04222F0700242F4014297
:10208C0042F0800223F824208BE70C7833F82420CC
:10209C0012F4804F0CD033F8242092B222F4E04298
:1020AC0022F0700242F4404242F0800223F82420D5
:1020BC000C7833F8242012F0400F0CD033F8242085
:1020CC0092B222F4E04222F0700242F4004242F05A
:1020DC00C00223F82420CA78012A1ED00C7833F8C9
:1020EC00242092B222F4E04222F0400282F020023C
:1020FC0042F4004242F0800223F82420097833F89D
:10210C00212092B222F4804222F0700242F400426A
:10211C0042F0800223F82120A7E70C7833F8242022
:10212C0092B222F4E04222F0400242F4004242F029
:10213C00800223F82420E1E70B7B002B46D14B785F
:10214C0013B30A7830F8223013F0400F0CD030F86B
:10215C0022309BB223F4E04323F0700343F400439A
:10216C0043F0C00320F822300A7830F822309BB2BA
:10217C0023F4E04323F0400343F4004343F0800393
:10218C0020F82230002070470A7830F8223013F4FF
:10219C00804F0CD030F822309BB223F4E04323F074
:1021AC00700343F4404343F0800320F822300A7854
:1021BC0030F822309BB223F4804323F0700343F4B5
:1021CC00004343F0800320F82230DBE74B78002BF0
:1021DC004ED10A7830F8223013F4804F0CD030F8FE
:1021EC0022309BB223F4E04323F0700343F44043CA
:1021FC0043F0800320F822300A7830F8223013F0B4
:10220C00400F0CD030F822309BB223F4E04323F083
:10221C00700343F4004343F0C00320F822300A78E3
:10222C0030F822309BB223F4E04323F0700343F4E4
:10223C00004343F0C00320F822300B7830F8232001
:10224C0092B222F4804222F0700248F2800C42EAF0
:10225C000C0220F823200A7830F822309BB223F4A9
:10226C00E04323F0400343EA0C0320F8223089E7D3
:10227C000A7830F8223013F4804F0CD030F822302A
:10228C009BB223F4E04323F0700343F4404343F048
:10229C00800320F822300A7830F8223013F0400FF7
:1022AC000CD030F822309BB223F4E04323F07003BF
:1022BC0043F4004343F0C00320F822300A7830F88E
:1022CC0022309BB223F4E04323F0700343F44043E9
:1022DC0043F0800320F822300B7830F8232092B2A0
:1022EC0022F4E04222F0400248F2800C42EA0C0256
:1022FC0020F823200A7830F822309BB223F4804354
:10230C0023F0700343EA0C0320F822303AE74B78B1
:10231C008BB10A7830F822309BB223F4E04323F0DF
:10232C00400383F0100343F4004343F0800320F890
:10233C002230002070470A7830F822309BB223F408
:10234C00804323F0700383F4805343F4004343F041
:10235C00800320F82230ECE70B7B002B4BD14B7821
:10236C0033B30A7830F8223013F0400F0CD030F829
:10237C0022309BB223F4E04323F0700343F4004378
:10238C0043F0C00320F82230CB78012B33D00A78ED
:10239C0030F822309BB223F4E04323F0400383F067
:1023AC00200343F4004343F0800320F8223022E062
:1023BC000A7830F8223013F4804F0CD030F82230E9
:1023CC009BB223F4E04323F0700343F4404343F007
:1023DC00800320F822300A7830F822309BB223F4A4
:1023EC00804323F0700383F4405343F4004343F0E1
:1023FC00800320F822300020704711B98023A0F808
:10240C004C30002070470020704700207047B0F817
:10241C00440080B270470020704710B45C1C640804
:10242C0000EB420202F5806207E00B78487843EA41
:10243C00002322F8043B0231013C002CF5D110BCE6
:10244C00704770B505460C464A78012A3BD00B7B89
:10245C00002B40F0A6828B690A69934240F2848279
:10246C009B1A8B61B5F850309BB22B44217803EB4F
:10247C000113B3F80C14C1F30901A3F80C143E2A90
:10248C0040F27682510912F01F0F00D10139B3F8D6
:10249C000C2492B2890289B20A4342F40042A3F896
:1024AC000C24227835F822309BB223F4804323F09D
:1024BC00700383F4405343F4004343F0800325F846
:1024CC002230002070BD8E6909698E4200D90E46FB
:1024DC00237B73B3E378022B4DD0236A9B1B2362BF
:1024EC00217835F8213013F0400F00F0F581002AE7
:1024FC0040F0E281B5F850309BB22B4403EB011352
:10250C00B3F80C24C2F30902A3F80C243E2E40F2BB
:10251C00BA81710916F01F0F00D10139B3F80C24E0
:10252C0092B2890289B20A4342F40042A3F80C2405
:10253C00CBE1B6B23346E28861692846FFF76DFFFE
:10254C00B5F850309BB22B44227803EB0213A3F85E
:10255C000464227835F822309BB223F4E04323F054
:10256C00400383F0300343F4004343F0800325F829
:10257C0022300020A6E7236A994280F066812278F7
:10258C0035F822309BB223F4E04323F0700343F47C
:10259C00014343F0800325F82230236A9B1B2362FE
:1025AC00227835F8223013F0400F00F0A7806378C2
:1025BC00B3BBB5F850309BB22B4403EB0213B3F80A
:1025CC000C24C2F30902A3F80C243E2E0FD9710976
:1025DC0016F01F0F00D10139B3F80C2492B2890206
:1025EC0089B20A4342F40042A3F80C241AE04EB913
:1025FC00B3F80C246FEA42426FEA524292B2A3F84B
:10260C000C240FE0720816F0010F00D00132B3F861
:10261C000C1489B2920292B20A43A3F80C2401E082
:10262C00012B30D0B3B2628961692846FFF7F5FE01
:10263C00636933446361236A226993422DD99B1BDE
:10264C0023626378002B45D1B5F850309BB22B44F4
:10265C00227803EB0213B3F80424C2F30902A3F8A3
:10266C0004243E2E1DD9710916F01F0F00D101391B
:10267C00B3F8042492B2890289B20A4342F40042AC
:10268C00A3F8042428E0B5F850309BB22B4403EB9C
:10269C000213B2B2A3F80C24C4E7002222621E4635
:1026AC00CFE74EB9B3F804246FEA42426FEA5242C4
:1026BC0092B2A3F804240FE0720816F0010F00D0B8
:1026CC000132B3F8041489B2920292B20A43A3F80D
:1026DC00042401E0012B06D0B3B22289616928469B
:1026EC00FFF79BFE35E7B5F850309BB22B442278B0
:1026FC0003EB0213B2B2A3F80424EDE76378B3BB87
:10270C00B5F850309BB22B4403EB0213B3F80424FE
:10271C00C2F30902A3F804243E2E0FD9710916F056
:10272C001F0F00D10139B3F8042492B2890289B287
:10273C000A4342F40042A3F804241AE04EB9B3F859
:10274C0004246FEA42426FEA524292B2A3F8042484
:10275C000FE0720816F0010F00D00132B3F8041428
:10276C0089B2920292B20A43A3F8042401E0012B2D
:10277C0030D0B3B2228961692846FFF74EFE6369F7
:10278C0033446361236A226993422DD99B1B2362D4
:10279C006378002B45D1B5F850309BB22B4422788E
:1027AC0003EB0213B3F80C24C2F30902A3F80C24B4
:1027BC003E2E1DD9710916F01F0F00D10139B3F847
:1027CC000C2492B2890289B20A4342F40042A3F863
:1027DC000C2428E0B5F850309BB22B4403EB0213C9
:1027EC00B2B2A3F80424C4E7002222621E46CFE74B
:1027FC004EB9B3F80C246FEA42426FEA524292B2DD
:10280C00A3F80C240FE0720816F0010F00D001326F
:10281C00B3F80C1489B2920292B20A43A3F80C24B6
:10282C0001E0012B06D0B3B2628961692846FFF73B
:10283C00F4FD8EE6B5F850309BB22B44227803EBB6
:10284C000213B2B2A3F80C24EDE7217835F821205D
:10285C0092B222F4E24222F0700242F4004242F0C0
:10286C00800225F82120B5F8502092B22A44217814
:10287C0002EB01129BB2A2F804342289616928464A
:10288C00FFF7CBFD65E64EB9B3F80C246FEA424274
:10289C006FEA524292B2A3F80C2416E0720816F0BA
:1028AC00010F00D00132B3F80C1489B2920292B22B
:1028BC000A43A3F80C2408E0B5F850309BB22B4423
:1028CC0003EB0113B2B2A3F80C24B3B262896169B1
:1028DC002846FFF7A2FD3CE6B2BBB5F850309BB2E0
:1028EC002B4403EB0113B3F80424C2F30902A3F83D
:1028FC0004243E2E0FD9710916F01F0F00D1013997
:10290C00B3F8042492B2890289B20A4342F4004219
:10291C00A3F8042421E04EB9B3F804246FEA424230
:10292C006FEA524292B2A3F8042416E0720816F031
:10293C00010F00D00132B3F8041489B2920292B2A2
:10294C000A43A3F8042408E0B5F850309BB22B449A
:10295C0003EB0113B2B2A3F80424B3B22289616968
:10296C002846FFF75AFDF4E500228A611A4679E5FC
:10297C004AB9B3F80C246FEA42426FEA524292B25F
:10298C00A3F80C248DE5510812F0010F00D0013191
:10299C00B3F80C2492B2890289B21143A3F80C1437
:1029AC007FE5CB78022B4DD0012B40F02F8189692C
:1029BC002369994240F2E680C91AA161F2B9B5F8CF
:1029CC00502092B22A44217802EB0112B2F804147E
:1029DC00C1F30901A2F804143E2B40F2D780580928
:1029EC0013F01F0F00D10138B2F8041489B2800221
:1029FC0080B2014341F40041A2F804146278002A29
:102A0C0040F0F680B5F8502092B22A44217802EBBF
:102A1C000112B2F80C14C1F30901A2F80C143E2BEC
:102A2C0040F2CD80590913F01F0F00D10139B2F8D3
:102A3C000C349BB2890289B20B4343F40043A2F8D5
:102A4C000C342EE5F2B9B0F850309BB203440A783E
:102A5C0003EB0213B3F80424C2F30902A3F8042411
:102A6C000A693E2A31D9510912F01F0F00D10139E0
:102A7C00B3F8042492B2890289B20A4342F40042A8
:102A8C00A3F804246378002B51D1B5F850309BB2D5
:102A9C002B44227803EB0213B3F80C24C2F3090283
:102AAC00A3F80C2422693E2A28D9510912F01F0FD1
:102ABC0000D10139B3F80C2492B2890289B20A43CD
:102ACC0042F40042A3F80C2433E04AB9B3F80424CE
:102ADC006FEA42426FEA524292B2A3F80424D1E761
:102AEC00510812F0010F00D00131B3F8042490B258
:102AFC008A0292B20243A3F80424C3E74AB9B3F89A
:102B0C000C246FEA42426FEA524292B2A3F80C24B0
:102B1C000FE0510812F0010F00D00131B3F80C2472
:102B2C0090B28A0292B20243A3F80C2401E0012B6A
:102B3C001DD0E369002B3FF4B4AC227835F8221099
:102B4C0044F2400303EA01008B4302D000287FF4D7
:102B5C00A8AC35F822309BB223F4E04323F0700389
:102B6C0043F4004343F0C00325F8223099E4B5F850
:102B7C0050309BB22B44227803EB0213228AA3F829
:102B8C000C24D6E70023A3610B4617E74BB9B2F828
:102B9C0004146FEA41416FEA514189B2A2F804145E
:102BAC002CE7590813F0010F00D00131B2F80404DE
:102BBC0080B2890289B20143A2F804141EE74BB912
:102BCC00B2F80C346FEA43436FEA53439BB2A2F85A
:102BDC000C3466E4590813F0010F00D00131B2F83F
:102BEC000C3498B28B029BB20343A2F80C3458E419
:102BFC00012A7FF456ACB5F8502092B22A442178C1
:102C0C0002EB01129BB2A2F80C344AE4012059E405
:102C1C0010B45C0800EB420000F5806007E030F86F
:102C2C00042B0A70C2F307224A700231013C002CBB
:102C3C00F5D113F0010F01D003880B7010BC704755
:102C4C0082B04FF0E0231B690193019BB0F1FF3F71
:102C5C0000D0013038B14FF0E0231B6913F4803FF2
:102C6C00F8D00138F6E702B070470000014B18604D
:102C7C00704700BF6800002010B504460E4B187852
:102C8C004FF47A73B3FBF0F30C4A1068B0FBF3F01B
:102C9C0000F08EF868B90F2C01D901200AE000224F
:102CAC0021464FF0FF3000F03DF8054B1C60002032
:102CBC0000E0012010BD00BF600000206800002073
:102CCC006400002008B5074A136843F01003136032
:102CDC00032000F015F80F20FFF7CEFFFDF74CFD99
:102CEC00002008BD00200240034A1168034B1B78EA
:102CFC000B441360704700BF6C1300206000002071
:102D0C00074AD36823F4E0631B041B0C000200F495
:102D1C00E060034343F0BF6343F40033D360704778
:102D2C0000ED00E000B5194BDB68C3F30223C3F1DF
:102D3C00070CBCF1040F28BF4FF0040C03F1040E78
:102D4C00BEF1060F18D9033B4FF0FF3E0EFA0CFCF8
:102D5C0021EA0C0199400EFA03F322EA030319430A
:102D6C0000280BDB0901C9B200F1604000F561409D
:102D7C0080F800135DF804FB0023E5E700F00F007A
:102D8C000901C9B2024B1954F4E700BF00ED00E091
:102D9C0014ED00E0002807DB00F01F0240090123BE
:102DAC009340024A42F82030704700BF00E100E037
:102DBC000138B0F1807F0BD24FF0E0235861054A07
:102DCC00F02182F823100020986107221A617047C5
:102DDC000120704700ED00E00C4B9A6803F580630E
:102DEC009B68134313F0010F0ED10B6833B142688B
:102DFC0022F470221343436000207047436823F48D
:102E0C00702343600020704701207047002401406C
:102E1C00836813F0010F0DD1436823F480734A6863
:102E2C0013434360836823F400630A68134383608D
:102E3C0000207047012070474B68826812F0010F28
:102E4C0023D110B4DBB1426822F468428C6823436E
:102E5C0013434360836823F4602323F481730A686B
:102E6C00CC6822430C692243134383604B68C26ACB
:102E7C0022F470021343C362002010BC70474268F6
:102E8C0022F4684213434360E4E7012070474A6828
:102E9C00836813F0010F1FD110B4B2B1436823F44F
:102EAC00A0538A68CC68224313434360836823F49D
:102EBC00E0430A68134383604B68826B22F4401230
:102ECC0013438363002010BC7047436823F4A05362
:102EDC00CA6813434360E9E701207047704798B113
:102EEC0008B50346D0F8B40210B10020C3F8B40200
:102EFC0009B1C3F8B012012183F89C121A7018465C
:102F0C00FDF7C2FD002008BD0220704719B1C0F8C2
:102F1C00B412002070470220704708B5FDF7F6FD8B
:102F2C00002008BD08B5D0F8B4322BB11B68984707
:102F3C0000B908BD0220FCE70220FAE708B5D0F87A
:102F4C00B4325B689847002008BD38B5044600F5DC
:102F5C002A75284600F035F90123C4F89432B4F8E8
:102F6C00AE32C4F8983294F8A81201F01F03012B6A
:102F7C000ED0022B11D02BB101F080012046FDF7B1
:102F8C00E0FD03E02946204600F0CAFA002038BDD7
:102F9C002946204600F0F8FAF8E72946204600F0CA
:102FAC0023FBF3E738B504460D4691BB1346D0F826
:102FBC009422032A03D0052A24D0084633E0D0F803
:102FCC006011D0F8642191420DD9891AC0F86011B2
:102FDC008A4206D98AB21946204600F037FC2846A8
:102FEC0021E092B2F7E7D0F8B4321B691BB190F82C
:102FFC009C22032A04D0204600F030FC284612E024
:10300C009847F8E70021C0F89412FDF79AFD28467E
:10301C0009E0D0F8B4329B6933B190F89C22032AB2
:10302C0004D19847002038BD0220FCE70220FAE7C3
:10303C0038B504460D46002953D11346D0F89422D6
:10304C00022A0CD0042A00D01AB980212046FDF7A0
:10305C0078FD94F8A032012B3ED0284638BD016A89
:10306C00426A91421BD8C169B1FBF2F302FB131304
:10307C002BB98A4203D8D0F8983299421CD3D4F891
:10308C00B432DB681BB194F89C22032A21D0802136
:10309C002046FDF756FD204600F0EBFBD9E78A1AD7
:1030AC00026292B2194600F0BAFB00231A46194686
:1030BC002046FDF77DFDCCE70022114600F0AFFB6A
:1030CC000021C4F898120B460A462046FDF770FD05
:1030DC00BFE720469847DAE7002384F8A032284659
:1030EC00BCE7D0F8B4325B6933B190F89C22032A68
:1030FC0004D198470020B1E70220AFE70220ADE7EA
:10310C0070B50446402300221146FDF707FD01254A
:10311C00C4F858514026C4F864613346002280211B
:10312C002046FDF7FBFCA561666284F89C520023E7
:10313C00C4F894326360C4F8A432D4F8B8322BB11A
:10314C00D4F8B4325B68002120469847002070BD4B
:10315C0001740020704790F89C3280F89D32042353
:10316C0080F89C320020704790F89C32042B01D0E0
:10317C000020704790F89D3280F89C32F8E708B533
:10318C0090F89C32032B01D0002008BDD0F8B4324B
:10319C00DB69002BF8D09847F6E70346002002E0E5
:1031AC000130C0B201331A78002AF9D1704708B542
:1031BC004B88012B00D008BDC0F8A43200F04EFBA8
:1031CC00F9E70B7803704B7843708B78CA7803EB74
:1031DC00022343800B794A7903EB022383808B799A
:1031EC00CA7903EB0223C380704710B504468021D3
:1031FC00FDF7A7FC00212046FDF7A3FC10BD30B560
:10320C0083B005460C460023ADF806304A88130AF5
:10321C00013B062B00F2A480DFE803F004182CA27B
:10322C00A2869300D0F8B0321B680DF10601007C29
:10323C009847BDF806201AB1E388002B40F0948023
:10324C00E388002B00F09A8003B030BD037C43B9B7
:10325C00D0F8B4329B6A0DF10600984702234370F4
:10326C00E7E7D0F8B432DB6A0DF106009847022389
:10327C004370DEE7D2B2052A52D8DFE802F0031021
:10328C001D2A3744D0F8B0325B6823B10DF106012A
:10329C00007C9847CDE72146FFF7A7FFD4E7D0F88D
:1032AC00B0329B6823B10DF10601007C9847C0E752
:1032BC002146FFF79AFFC7E7D0F8B032DB6823B19D
:1032CC000DF10601007C9847B3E72146FFF78DFF0F
:1032DC00BAE7D0F8B0321B6923B10DF10601007CBE
:1032EC009847A6E72146FFF780FFADE7D0F8B0324C
:1032FC005B6923B10DF10601007C984799E72146E3
:10330C00FFF773FFA0E7D0F8B0329B6923B10DF142
:10331C000601007C98478CE72146FFF766FF93E790
:10332C002146FFF762FF8FE7037C33B9D0F8B43244
:10333C005B6B0DF1060098477BE72146FFF755FFC5
:10334C0082E7037C43B9D0F8B4321B6B0DF1060055
:10335C009847072343706CE72146FFF746FF73E756
:10336C002146FFF742FF6FE79A4228BF1A46ADF895
:10337C0006200146284600F045FA61E7284600F091
:10338C006DFA61E738B504468B88F3B9CB88E3B99D
:10339C004B887F2B19D803F07F0590F89C32032BB8
:1033AC000CD080F89E522946FDF7F2FB204600F027
:1033BC0055FA35B1022384F89C3209E0FFF715FF6A
:1033CC0006E0012384F89C3202E02046FFF70DFF53
:1033DC0038BD000038B504460D468978284B197065
:1033EC0001290ED890F89C32022B0ED0032B21D041
:1033FC002946FFF7FAFE224B19782046FFF79EFD6F
:10340C0002E02946FFF7F1FE38BD81B1416003238C
:10341C0080F89C32FFF786FD022803D0204600F08E
:10342C001DFAF1E729462046FFF7DFFEECE700F036
:10343C0015FAE9E789B1436899421DD0D9B2FFF773
:10344C007DFD0F4B197861602046FFF76BFD02285C
:10345C000DD0204600F002FAD6E7022380F89C3209
:10346C004160FFF76BFD204600F0F8F9CCE72946E8
:10347C002046FFF7BAFEC7E700F0F0F9C4E700BF3B
:10348C007013002008B5CB88012B0AD190F89C3220
:10349C00022B09D9032B09D10122011D00F0B2F92D
:1034AC0001E0FFF7A2FE08BD5BB213B9FFF79DFE6A
:1034BC00F9E70146002341F8083F012200F0A2F988
:1034CC00F1E708B590F89C32013B022B12D8CB885F
:1034DC00022B0CD10123C360D0F8A4320BB103230F
:1034EC00C360022200F10C0100F08CF908BDFFF75B
:1034FC007CFEFBE7FFF779FEF8E708B590F89C3205
:10350C00013B022B09D84B88012B00D008BD0023AE
:10351C00C0F8A43200F0A2F9F8E7FFF766FEF5E771
:10352C0008B50B7803F06003202B05D0402B03D09B
:10353C0043B1FFF75AFE03E0D0F8B4329B689847CA
:10354C00002008BD4B78092B1BD8DFE803F01117BE
:10355C001A141A08051A0E0BFFF751FEF0E7FFF7C5
:10356C0011FFEDE7FFF736FFEAE7FFF78BFFE7E721
:10357C00FFF7A7FFE4E7FFF71AFEE1E7FFF7BDFF50
:10358C00DEE7FFF732FEDBE738B505460C460B7875
:10359C0003F06003202B06D0402B04D01BB1FFF7A7
:1035AC0024FE002038BD95F89C32013B022B16D826
:1035BC002379012B0ED8D5F8B4329B6821462846C6
:1035CC009847E388002BECD10028EAD1284600F07C
:1035DC0045F9E6E721462846FFF707FEE1E72146D5
:1035EC002846FFF702FEDCE770B505468B880C78A1
:1035FC0004F06004202C07D0DAB2402C04D05CB16B
:10360C00FFF7F3FD002405E0D5F8B4329B6828469B
:10361C0098470024204670BD202C09D04E78012EEE
:10362C0033D0032E0AD0002E55D0FFF7DEFDF1E784
:10363C00D0F8B4329B6898470446EBE790F89C327C
:10364C00022B04D0032B11D0FFF7CFFDE2E70AB118
:10365C00802A03D12846FFF7C8FDDBE71146FDF7AA
:10366C0070FA80212846FDF76CFAD3E74B8823B912
:10367C001AB1802A01D0CB881BB1284600F0EEF895
:10368C00C8E71146FDF75DFAF7E790F89C32022B7C
:10369C0004D0032B11D0FFF7A8FDBBE70AB1802A99
:1036AC0003D12846FFF7A1FDB4E71146FDF749FA0F
:1036BC0080212846FDF745FAACE74B88002BA9D1B1
:1036CC0012F07F0F03D1284600F0C8F8A2E711468C
:1036DC00FDF73FFAF7E790F89C02022806D0032882
:1036EC0029D02846FFF781FD344693E70AB1802A9A
:1036FC0013D113F0800F15D102F07F0202EB82027E
:10370C00910001F5A8712944043100230B600222B9
:10371C00284600F077F834467CE72846FFF765FD2D
:10372C00344677E702F07F0202EB820291001031FF
:10373C0029440431E9E75BB2002B1FDB02F00F00D8
:10374C0000EB800005EB8000D0F8580120B3002B73
:10375C0027DB02F07F0303EB83039C0004F5A874C2
:10376C002C4404340AB1802A24D100232360022281
:10377C002146284600F046F834464BE702F00F008D
:10378C0000EB800005EB800080690028DFD1284623
:10379C00FFF72BFD34463DE72846FFF726FD344660
:1037AC0038E702F07F0303EB83039C0010342C44B6
:1037BC000434D7E711462846FDF7D3F910B101239D
:1037CC002360D4E700232360D1E7D0B170B50D4658
:1037DC0016460446FFF7E1FC431C5B009BB23380AA
:1037EC002B7003236B70022307E001345A1CD2B2F6
:1037FC00E8540233DBB20021A95420780028F4D11C
:10380C0070BD704708B513460222C0F89422C361FC
:10381C0003620A460021FDF7C3F9002008BD08B574
:10382C0013460A460021FDF7BBF9002008BD08B578
:10383C0013460322C0F89422C0F85C31C0F8603102
:10384C000A460021FDF7B4F9002008BD08B513465F
:10385C000A460021FDF7ACF9002008BD08B5042389
:10386C00C0F8943200231A461946FDF799F9002046
:10387C0008BD08B50523C0F8943200231A46194632
:10388C00FDF796F9002008BD10B5D0F8B842D0F875
:10389C00BC325BB194F80002FF2807D09B6894F807
:1038AC00012221469847FF2384F80032002010BDE6
:1038BC004323038000487047A40000204323038067
:1038CC0000487047E80000204323038000487047FD
:1038DC00380100200A230380004870472C01002087
:1038EC0038B50446D0F8B852FDF76AF9C5F80C02A1
:1038FC00D4F8B8324BB1D4F8BC32DB6805F503719F
:10390C00D5F804029847002038BD0220FCE710B51A
:10391C00D0F8B822D0F8C042F2B101EB810300EB31
:10392C008303DB694BB101EB810C04EBCC04A46B7E
:10393C00B3FBF4FC04FB1C3323B10023C2F8143298
:10394C00002010BD01EB810300EB83030022DA6140
:10395C001346FDF725F9F3E70220F2E7F0B583B043
:10396C0006460C46D0F8B87200238DF80730ADF837
:10397C0004300B7813F0600527D0202D53D1CA8862
:10398C00DAB113F0800F0CD0D0F8BC329B683946FA
:10399C0060789847E28839463046FFF733FF0025B8
:1039AC0044E04B7887F800328B7987F80132CA886B
:1039BC003946FFF73CFF002538E0D0F8BC329B6855
:1039CC00002248789847002530E04F780A2F14D011
:1039DC000B2F20D01FB1FFF708FC022526E090F832
:1039EC009C32032B03D0FFF700FC02251EE00222C1
:1039FC0001A9FFF707FF3D4618E090F89C32032B16
:103A0C0003D0FFF7F2FB022510E001220DF10701B4
:103A1C00FFF7F8FE0AE090F89C32032B06D0FFF774
:103A2C00E4FB022502E0FFF7E0FB0225284603B089
:103A3C00F0BD38B504468121FDF77BF80025E56221
:103A4C0001212046FDF775F8C4F86C5182212046FF
:103A5C00FDF76FF82564D4F8B8324BB1D4F8BC320A
:103A6C005B689847D4F8B802FDF7B4F8C4F8B852BC
:103A7C00002038BD70B50446037CABBB4FF400731B
:103A8C0002228121FDF74AF80125E5624FF400730B
:103A9C00022229462046FDF741F8C4F86C51082350
:103AAC00032282212046FDF739F8012323644FF4C9
:103ABC000770FDF78BF80546C4F8B80268B3D4F864
:103ACC00BC321B6898470023C5F81432C5F818326D
:103ADC00267CCEB94FF40073D5F804220121204680
:103AEC00FDF766F8304670BD402302228121FDF7B8
:103AFC0015F80125E5624023022229462046FDF7F0
:103B0C000DF8C4F86C51CAE74023D5F80422012102
:103B1C002046FDF74DF80026E4E70126E2E719B14F
:103B2C00C0F8BC120020704702207047D0F8B832A1
:103B3C00C3F80812C3F8102200207047D0F8B8322E
:103B4C00C3F8041200207047D0F8B82292B108B51F
:103B5C00037C43B94FF40073D2F804220121FDF722
:103B6C0027F8002008BD4023D2F804220121FDF7DC
:103B7C001FF8F6E70220704730B4036A23F0010304
:103B8C000362036A4468826922F073020D682A4357
:103B9C0023F002030D692B4323F001034D682B43E3
:103BAC000F4DA84207D044608261CA684263036229
:103BBC00002030BC704723F008034D6943EA8503AD
:103BCC0023F004038D6843EA850324F480748D6923
:103BDC002C4324F40074CD6944EA4504E3E700BFA8
:103BEC00002C014030B4036A23F010030362036A13
:103BFC004468826922F4E6420D6842EA052223F009
:103C0C0020030D6943EA051323F010034D6843EAC2
:103C1C000513104DA84207D044608261CA688263C4
:103C2C000362002030BC704723F080034D6943EAE7
:103C3C00851323F040038D6843EA851324F48064D4
:103C4C008D6944EA850424F40064CD6944EAC50412
:103C5C00E2E700BF002C014030B4036A23F4807308
:103C6C000362036A4468C26922F073020D682A4336
:103C7C0023F400730D6943EA052323F480734D6824
:103C8C0043EA05230F4DA84207D04460C261CA68BD
:103C9C00C2630362002030BC704723F400634D699B
:103CAC0043EA852323F480638D6843EA852324F457
:103CBC0080548D6944EA051424F40054CD6944EA17
:103CCC004514E2E7002C014030B4036A23F480531E
:103CDC000362036A4468C26922F4E6420D6842EA50
:103CEC00052223F400530D6943EA053323F4805372
:103CFC004D6843EA0533084DA84207D04460C261C1
:103D0C00CA6802640362002030BC704724F480440B
:103D1C008D6944EA8514F1E7002C014003681A4AC6
:103D2C0090420AD0B0F1804F07D0A2F59432904265
:103D3C0003D002F58062904203D123F070034A68ED
:103D4C001343114A90420AD0B0F1804F07D0A2F52C
:103D5C009432904203D002F58062904203D123F456
:103D6C004073CA68134303608B68C3620B88836219
:103D7C00054B984205D0436943F001034361002091
:103D8C0070470B690363F6E7002C014008B50B463E
:103D9C001146B3F5807F14D008D8012B0ED0102B10
:103DAC0002D1FFF71FFF08E0012006E0B3F5805FAA
:103DBC0002D1FFF789FF00E0012008BDFFF7DCFE10
:103DCC00FBE7FFF749FFF8E70B7B8A68134323F403
:103DDC0080634A68134323F400630A68134323F493
:103DEC008053CA89134323F400530A69134323F401
:103DFC0080434A691343436400207047FFF76EF811
:103E0C000B480C490C4A002302E0D458C45004332C
:103E1C00C4188C42F9D3094A094C002301E0136001
:103E2C000432A242FBD300F00FF8FCF777FC70478A
:103E3C00000000207C010020243F00087C010020B1
:103E4C0074130020FEE7000070B500260C4D0D4CDD
:103E5C00641BA410A64209D100F022F800260A4DDA
:103E6C000A4C641BA410A64205D170BD55F8043B46
:103E7C0098470136EEE755F8043B98470136F2E7D0
:103E8C001C3F00081C3F00081C3F0008203F000896
:103E9C0003460244934200D1704703F8011BF9E733
:103EAC00F8B500BFF8BC08BC9E467047F8B500BF1B
:083EBC00F8BC08BC9E467047EB
:103EC40000000800000008000000000004040400D2
:103ED40053544D3332205669727475616C20436FAC
:103EE4006D506F727400000053544D6963726F65B6
:103EF4006C656374726F6E6963730000434443209E
:103F0400436F6E666967000043444320496E7465DD
:083F14007266616365000000A4
:043F1C007501000823
:043F20004D01000847
:103F24001D08000829080008ED080008C908000851
:103F3400B5080008090900082D090008120100024B
:103F44000202004083044057000201020301000002
:103F5400040309041A03000000000000000000002C
:103F6400000000000000000000000000000000004D
:103F74007D0900085109000855090008590900087D
:103F840001000000100000000024F400813A000841
:103F94003F3A00086939000800000000953800081D
:103FA4001B390008ED380008000000000000000084
:103FB40000000000C9380008BD380008D5380008E2
:103FC400E138000809024300020100C0320904007C
:103FD4000001020201000524001001052401000172
:103FE40004240202052406000107058203080010C8
:103FF40009040100020A0000000705010240000054
:10400400070581024000000009024300020100C0CC
:104014003209040000010202010005240010010518
:10402400240100010424020205240600010705827C
:104034000308001009040100020A0000000705013A
:104044000200020007058102000200000A060002C5
:10405400000000400100000009074300020104C001
:1040640032090400000102020100052400100105C8
:10407400240100010424020205240600010705822C
:104084000308001009040100020A000000070501EA
:0C4094000240000007058102400000000F
:0400000508003E09A8
:00000001FF
